:020000020000FC
:100000004DC0FFB6989B39C01123B1F4B29B29C0F3
:020010000AC024
:10001600FFB6112789B3807F8BBB882789BF37C07E
:10002600962CA72CB82C662477248824CC24DD248F
:10003600EE24B29B07C013959EEC92BF81E088BF69
:1000460081E089BF123060F069F0143020F031F49D
:100056009091690008C09B2D906205C0992703C046
:10006600992D01C09A2DB29992959F7089B3807F80
:10007600982B08C099B3907FB29B03C08FEF9F6007
:1000860002C09229812D9BBB88BB92E0B29B93E074
:1000960095BFFFBE189521E02EBF2FE52DBF2FEF90
:1000A6002ABB2BE027BB20E42BBF23E023BFB9D319
:1000B60060E085D26DD2F8946FEF81D22FEF28BB26
:1000C6002BBB66D2222723BB20936800B7D380F3CD
:1000D60060E075D200FDD9D001FDE8D002FD39D12E
:1000E60004FDD8D005FDF0D0202F2295022B6624E2
:1000F6007724882455243324442413D093E095BFD1
:1001060078944DD2889400FD36D040F001FD43D05E
:1001160028F002FD20D010F004D0F2CF2E3081F767
:10012600CACF98990BC0242D6FEF26272F70222E49
:1001360069B3607F262BB29B2BBB03C06C2C7D2C36
:100146008E2C232D25296FEFB29968BB2627B29BEB
:1001560028BB122E089520916E002A9519F020933F
:100166006E00089520917B0020936E00A2D2C8F302
:10017600C1F3A9D11FC020916E002A9519F02093D2
:100186006E00089520916C0020936E0092D2C8F301
:10019600C1F366D10FC020916F002A9519F0209304
:1001A6006F00089520916D0020936F007DD2C8F3F3
:1001B600C1F303D0989488940895989A2091680082
:1001C60021FD9898B0E0A9E822E099992D91233075
:1001D60008F008952D91662720FD626021FD61607B
:1001E600562E2695269536D0209369009B992D91FB
:1001F6009C9911C09A9918C0CD90DD902D912AD066
:100206002F70E22E2C2D219525D0C22E2D2D219535
:1002160021D0D22E08956D912D9129D0C62E6D91A3
:100226002D9125D0D62EEACF6D912C912F7023FDDE
:10023600206F1DD0C62E6D9162956F705C915295A0
:10024600507F652B2D9122952F7023FD206F0FD0A7
:10025600D62ED4CF222351F0622F2A7A60FD246055
:1002660062FD216064FD206466FD2061089527FD1E
:1002760006C0222311F467FF08956FE708952F3F04
:1002860011F467FD089560E8089520917900509172
:100296007B0004C020917A0050917C0020936A0074
:1002A60050936C0050936E0020E0D5C020917900E9
:1002B60020936B0020917B0020936D0020936F00AC
:1002C60060917D0016D20DC020917A0020936B00BC
:1002D60020917C0020936D0020936F0060917E003A
:1002E60005D209F0089550917400A1E8B0E05523B5
:1002F600F9F05A952D91253821F4999A5A952D9110
:10030600F6CF253931F45A952D91203181F79B9AF4
:10031600EECF253739F45A952D91203131F02C3016
:1003260031F0E5CF06D019F308959C9A08959A9A6C
:100336000895237061F02A9539F02A9511F0989462
:1003460008955A95E1F32D915A95C9F32D91189474
:100356000895222720937F002091790020936A0038
:1003660020917B0020936C0020936E0060917D00AD
:10037600C0D121F0089505010904A101509174002E
:10038600A1E8B0E0ECE7F3E036E005902D9120150A
:1003960089F75A953A95C9F733275A952D912538F5
:1003A60021F433955A952D91F8CF213A21F45A9597
:1003B6002D91223011F0989408955A952D91253754
:1003C600D1F75A952D912830B1F75A952D912537A9
:1003D60019F1253911F40CD0F8CF293011F40BD0CE
:1003E600F4CF213811F411D0F0CFA3DF71F30895C3
:1003F6005A950D9008955A952D910A943395203368
:1004060009F0089530937F0008955A952D91213073
:1004160009F00895300D08955A952D91213019F05F
:10042600243059F008955A952D91253909F00895EB
:100436005A952D91243009F001C030683093800020
:100446001894089560918300693309F0089562E075
:100456002091680026272093680021FD9898E6C021
:10046600F1DFB0E0A1E860E02C912F7009F061E0C7
:100476002D91207F09F062E0362E2D9133276627D5
:1004860008D0622BA938E0F3462E232D232B322EDB
:1004960008955D912227583591F05A3291F05C32D9
:1004A60071F028E05F5451F021E05A9539F022E0CE
:1004B6005A9521F024E05A9509F0222708953260D2
:1004C60008953160089520917F00222309F02FC0FE
:1004D600209182002F3739F02091860025952295AC
:1004E6006091870009C0209186002F702F30A1F3FC
:1004F60020918600622F2295262B2370662720FDE9
:10050600626021FD6160362E60E02091850020301A
:1005160009F464602F3F09F4626020918400203062
:1005260009F461602F3F09F46860462E08952A9504
:10053600B0E0A1E8A20F66272D91203009F4616092
:100546002F3F09F468602D91203009F464602F3F35
:1005560009F46260462E20918000622F6F77A1E831
:10056600A60F6D915C9127FF08C056956795569525
:1005760067955695679556956795562F5295679543
:10058600652B222760FD226061FD2160322E0895D1
:1005960032E303D03A95E9F7089544E601C04AE00C
:1005A60003D04A95E9F7089524E60000000000000C
:1005B600000000002A95C9F7089523E0F6CF78EAEF
:1005C6007260DF987FB920D06FB91ED0DF9A089588
:1005D6007260DF987FB918D02D9115D05A95E1F742
:1005E600DF9A0895DF987FB90FD0222715D0DF9ABA
:1005F6000895DF987FB908D022270ED02D935A95FB
:10060600D9F7DF9A08952FB920E42EB93BE13DB919
:100616002EB126FFFCCF08952FB920E42EB93BE179
:100626003DB92EB126FFFCCF2FB10895F9E0E6E8DB
:1006360061E083D170E258E0CBDF60E478EEC0DFA2
:1006460020E120937000B4D009F0089560E878EEB8
:10065600B7DF2227209371002093720003C060E069
:1006660078E3AEDF6091680070E1AADF61E078E3CD
:10067600A7DF20E220937000C6D009F40895243045
:1006860041F420917100239520937100283C39F79D
:1006960009C02E3039F42091720023952093720000
:1006A6002530E9F622230895A9E8B0E020916B00F1
:1006B60004C0A1E8B0E020916A0020937000A3D0A6
:1006C60029F0243011F008940895089570E38ADF24
:1006D600522F2F9378E086DF2D935A95D9F778EC31
:1006E60064E06EDF2F91222388940895F9E0E6EA0C
:1006F60009C0F9E0EEE906C0F9E0E6E903C062E107
:10070600F9E0EEE81AD170E258E062DF20E12093CA
:1007160070004ED009F0089578EE60E2609377009D
:100726004FDF2E912E9106D021F420EA20937000FF
:100736003FC00895A1E8B0E02093760022272093D9
:10074600740020E02093700033D009F0089570E320
:1007560049DF20937300522F78E044DF2D935A959A
:10076600D9F778EC64E02CDF209174005091730087
:10077600250F2093740020917500521730F02091B8
:100786007400509176002517E0F222270895F9E0CB
:10079600EEE7D2D0A0E6B0E070E258E019DF20E143
:1007A6002093700005D009F0089520E8209370008A
:1007B6002227209371002093720025D009F4089512
:1007C600243041F420917100239520937100283C38
:1007D600A1F709C02E3039F4209172002395209399
:1007E6007200253051F7263061F460917700603150
:1007F60011F060E101C060E26093770078EEE0DE20
:10080600E1F6222308956091700070EFD9DE78EC4E
:10081600E9DE2078E1F360E8D3DE78EFE3DE2F70DF
:10082600089578E864E1CCDE78E760E2C9DE60E04E
:10083600C7DE78E6D7DE2170E9F3089535D090F16A
:1008460058EC86D04CD071F55ADF61F568E054DF7C
:1008560049F56091830050DF30918500EAE8F0E0C9
:100866000781002309F404E0208920937D00248970
:100876002F7020937900208D20937B00313079F002
:10088600E3EAF0E027812295022B208920937E005F
:1008960024892F7020937A00208D20937C0077DFA7
:1008A600889408950894089578ED61EC89DE78ECD3
:1008B60060E286DE78EE64E083DE78EF93DE207C0D
:1008C60061F078ED203821F06BEC7ADE189403C0E5
:1008D60069EC76DE9894889408950894089528E043
:1008E6002093750078EE61E06BDE78EE7BDE21709A
:1008F600E1F758EC2DD060E070EE62DE68E000DFD4
:1009060009F00895209188002093750078EE61E043
:1009160057DE78EE67DE2170E1F758EC19D0F9E082
:10092600EEE637DF09F008955EE112D061E070EE81
:1009360047DEF9E0E6E72DCF662707D058E0259198
:100946002D935A95E1F75E936E93B0E0A0E6089575
:1009560078EC60E435DE78EC45DE2074E1F360E4A3
:100966002FDE5A95C1F7089500050100000000002A
:100976000009010000000000210A0000000000003C
:10098600210900020000010080060001000012009B
:100996008006000200008000810600220000800020
:0809A60081060022010080001F
:100FC0004D756C746948494431207665722E322E15
:100FD0003420202033302E31322E323032300D0A80
:100FE000415454696E7934342F3834202020202025
:100FF000202020202020286329206361726F0D0AA1
:00000001FF
